:020000040000FA
:02000000A8282E
:080008000D2852346534613407
:10001000643479340D340A3400348B138B1B0D286F
:100020008C008C0E8316010E8E008312030E8D0041
:100030008B1826280B1924280D0E830083160E0E0C
:10004000810083120C0E09000B1187280108920011
:1000500003308100920E921986280730120582071C
:100060008628382886283D28432886284B28482873
:10007000930D931C862813105428930D931C131072
:10008000931813145428930D931886281314542886
:100090001614961D5228961D86280D30D2200A303F
:1000A000D22086288B101C28161C8628940A961CA1
:1000B0006428161D7528941D63289401950A130859
:1000C0009900B7209615522804301402031D6328A6
:1000D0009401130897000F301705970096149A00A3
:1000E000B7202030D2209A0A632805301402031D5D
:1000F00063289401130898001F3098051808B7204A
:100100009A0B63282030D220161563288B100130FB
:1001100093009401960195019701980199011C287B
:100120008316013086001F3085008316063081005B
:1001300083128601033081000130930094019601FF
:100140009501970198019901B0308B008614080041
:100150009020FF30E6200530AE20AD289000B6207C
:10016000003803190800D220100AAE28820090003F
:10017000100E0F39C120D22010080F39C120D22013
:100180000800820730343134323433343434353477
:1001900036343734383439344134423443344434D7
:1001A000453446348610910008308F000608111837
:1001B0000238111CFD398600910C8F0BD7280000E6
:1001C0000000000000000000861402308F008F0B3A
:0401D000E728080014
:02400E00F23F7F
:00000001FF
